:1000000083C111C09AC199C1DAC197C196C195C186
:1000100094C193C192C191C190C18FC18EC18DC154
:100020008CC18BC18AC1CF93CFB7CF93C395819B2E
:10003000E9F7819B09C0819B07C0819B05C0819B1B
:1000400003C0819B01C0A3C0DF93C0918400DD2762
:10005000C557DF4F819B02C0DF91EBCF2F930F93EA
:100060001F9300B32FEF01FB20F94F933F9310B381
:100070004FEF012701FB21F93BE031C04E7F012FFB
:1000800010B3216028C0102F4D7F2260000000B304
:1000900029C04B7F2460012F000010B32BC010B388
:1000A000477F28602AC04F7E00B320612CC04F7D5F
:1000B00010B320622FC04F7B00B3206432C04227B0
:1000C00000B349934FEF0000102711FB20F910B344
:1000D0001670C9F1297F91F2012701FB21F900B3C4
:1000E000237F89F2315058F1102711FB22F910B308
:1000F000277E79F2012701FB23F92F7C81F200B3DF
:10010000102711FB24F92F7971F200C010B30127D9
:1001100001FB25F92F7359F200C000B3102711FB22
:1001200026F9223040F200C010B3012701FB27F965
:10013000243028F64F77206810B30000F9CF10E480
:100140001ABF002719C03B503195C31BD04010E4A3
:100150001ABF0881033CF9F00B34E9F020918200CA
:100160001981110F1213EDCF4A81441F093641F155
:100170000D3211F0013E29F7009389003F914F9114
:100180001F910F912F91DF91CAB7C6FD4FCFCF912D
:10019000CFBFCF91189520918900222379F3109138
:1001A0008700112369F534306AF13093870020937A
:1001B0008300109184003BE0311B3093840022C007
:1001C000009187000130E4F40AE54F7049F4309162
:1001D000620034FD19C000936200CBE6D0E018C085
:1001E0003091760034FD10C000937600C7E7D0E070
:1001F0000FC02795A8F45150A9F4220F0000F9CFA1
:100200004AE503C042ED01C0432FC4E1D0E032E033
:1002100011B31660919A11BB02B320E416E05F930C
:10022000012756E002BB279520F4515021F4220FFC
:10023000F9CF012756E000003B5A02BBD0F22795C8
:1002400028F4515029F4220F0000F9CF012756E07D
:10025000279502BB20F4515021F4220FF9CF01273A
:1002600056E02991332302BB21F6097F10918800C3
:10027000110FC651D04002BB11F01093820010E460
:100280001ABF026011B3197F402F497F5F9100C0F0
:1002900000C002BB11BB42BB71CF040309041003B1
:1002A0004300540048004E002E0064006500100317
:1002B0004C004500440043007500620065001201D7
:1002C000100100000008C016DF0500010102000156
:1002D00009022200010100807D09040000010300E1
:1002E0000000092101010001221600070581030811
:1002F000000A0600FF0901A101150026FF0075088C
:1003000095010900B20201C011241FBECFEDCDBF7F
:1003100010E0A0E6B0E0E4EEF7E002C005900D9238
:10032000A436B107D9F710E0A4E6B0E001C01D92F1
:10033000A13AB107E1F72ED053C262CEA82FB92F50
:1003400080E090E041E050EA609530E009C02D91F6
:1003500082279795879510F084279527305EC8F3FC
:100360006F5FA8F30895EADF8D939D9308958FEF53
:1003700087BB88BB88E781BB80E482BB89B7806488
:1003800089BF82E08BBD81E78ABD8EB58B608EBD53
:1003900078940895ECDFE0D184D0FECF90E0880F10
:1003A000991F880F991F80509040F2D1609366008A
:1003B00070936700809368009093690008951F927E
:1003C0000F920FB60F9211242F933F934F935F9389
:1003D0006F937F938F939F93AF93BF93EF93FF930D
:1003E000809165008150809365008823C9F48091D5
:1003F0006A0090916000803239F4913011F41092CB
:10040000600010926A0008C0992331F0C7DF809124
:100410006A008F5F80936A0080916100809365001D
:1004200082B3877882BB92B390648091640028E0A5
:1004300030E0082E02C0220F331F0A94E2F7922BFD
:1004400092BB69E09CD12091660030916700409199
:1004500068005091690004C05695479537952795D7
:100460008A95D2F7822F809588BB30FD969880912F
:1004700064008F5F80936400833010F010926400FA
:10048000FF91EF91BF91AF919F918F917F916F916C
:100490005F914F913F912F910F900FBE0F901F9042
:1004A00018951F93CF93DF9380918700835087FD2A
:1004B000A1C090918400209183002D3209F098C052
:1004C000883009F095C0CCE0D0E0C91BD109C557F0
:1004D000DF4F83EC80936B008AE58093620013BA50
:1004E0008881807619F0CE01DBD079C09A81109294
:1004F00074008981882331F41092750024E730E07C
:1005000082E069C0853019F49093880061C086301C
:1005100009F048C08B81813041F48EEB92E09093DA
:1005200086008093850082E13AC0823041F480EDFC
:1005300092E0909386008093850082E230C0833001
:10054000C9F4992341F48AE992E09093860080935C
:10055000850084E024C0913019F48EE992E004C053
:100560009230E1F48EEA92E09093860080938500C9
:1005700080E115C0813241F482EE92E090938600D2
:100580008093850089E00BC0823241F482EF92E0D3
:10059000909386008093850086E101C080E090E41E
:1005A00093BB1DC0883069F0893019F490938A009C
:1005B0000FC08A3049F08B3059F48BE48093770078
:1005C00007C02AE830E002C024E730E081E003C041
:1005D00024E730E080E030938600209385009F81FF
:1005E000992321F49E81981708F4892F8093630042
:1005F000109287008091620084FF44C08091630064
:100600008F3F09F43FC0182F893008F018E0811B94
:100610008093630080916B0098E8892780936B003A
:10062000112321F1E0918500F0918600812F815006
:100630009E9B0CC090E083599F4FACE6B0E02491A4
:100640002D933196A817B907D1F70CC0EF0190E0B0
:1006500083599F4FACE6B0E029912D93FE01A81776
:10066000B907D1F7F0938600E09385008CE690E01F
:10067000612F79DE1C5F1C3019F08FEF80936300CF
:100680001093620084E190B3967031F48150D9F7F1
:100690001092880010928200DF91CF911F910895EF
:1006A000FC0180818076803409F054C081818130E2
:1006B00091F5848173816281209166003091670099
:1006C0004091680050916900882359F4972F80E089
:1006D000860F911DAA2797FDA095BA2F2070307024
:1006E0000DC0972F80E0860F911DAA2797FDA0953A
:1006F000BA2FDC019927882740705070822B932BEA
:10070000A42BB52B8093660090936700A09368009C
:10071000B09369001FC0823091F4848190E0880F0B
:10072000991F880F991F4091660050916700609152
:10073000680070916900805090402DD00BC08430CB
:1007400021F482818093610005C0833019F4828195
:100750008093600080E0089585B7826085BF8BB785
:1007600080648BBF8BE4809377008AE5809376006A
:10077000899A01C000009150E9F7899808950024F2
:1007800080FD060E660F11F08695D1F7802D089535
:10079000A6E144E00AC0242F16D0252F14D000C0B3
:1007A00011D0272F10C0A82F862FE82FE199FECF58
:1007B0001FBA05C0EEBBE09AE3950DB20D92415011
:1007C000C8F70895262FE199FECF1CBA1FBA8EBB39
:1007D0002DBB0FB6F894E29AE19A0FBE01960895E8
:0407E000F894FFCFBB
:0407E400020A5AFFAC
:00000001FF
